:020000040800F2
:1000000028360020E9020008DB26000875240008D5
:10001000D9260008290700086D33000800000000F9
:10002000000000000000000000000000290200089D
:10003000E707000800000000850200083F290008CB
:100040000303000803030008030300080303000878
:100050000303000803030008030300080303000868
:1000600003030008030300080303000885070008D2
:1000700091070008030300080303000803030008B6
:100080000303000803030008030300080303000838
:100090000303000803030008030300080303000828
:1000A0000303000803030008030300080303000818
:1000B0000303000800000000000000000303000824
:1000C0000303000803030008030300080000000006
:1000D000030300080303000803030008613300085A
:1000E00003030008030300080303000800000000E6
:1000F0000000000000000000000000000000000000
:1001000000000000000000000000000003030008E1
:1001100000000000000000000303000800000000D1
:1001200000000000000000000000000000000000CF
:1001300000000000000000000000000000000000BF
:100140000303000803030008000000000000000093
:10015000000000000000000000000000000000009F
:100160000303000803030008030300080303000857
:100170000303000800000000000000000000000071
:10018000000000000303000800F002F800F03CF853
:100190000AA090E8000C82448344AAF10107DA45E2
:1001A00001D100F031F8AFF2090EBAE80F0013F0F8
:1001B000010F18BFFB1A43F001031847F450000069
:1001C00014510000103A24BF78C878C1FAD85207F9
:1001D00024BF30C830C144BF04680C6070470000C1
:1001E0000023002400250026103A28BF78C1FBD840
:1001F000520728BF30C148BF0B6070471FB504F0DD
:10020000A5FF1FBD10B510BD00F0D0F91146FFF7D6
:10021000F5FF03F007F900F0EEF903B4FFF7F2FF82
:1002200003BC00F0F5F900002C4B19680868B0E831
:10023000F04F80F30988BFF36F8F4FF0000080F319
:10024000118870470000000008480068006880F3CB
:1002500008884FF0000080F3148862B661B6BFF3DF
:100260004F8FBFF36F8F00DF00BF00BF08ED00E0CE
:10027000DFF80C00016841F470010160704700BFB5
:1002800088ED00E0EFF30980BFF36F8F134B1A681E
:100290001EF0100F08BF20ED108A20E9F04F10600B
:1002A00009B44FF0500080F31188BFF34F8FBFF3B4
:1002B0006F8F04F09FF94FF0000080F3118809BCA4
:1002C00019680868B0E8F04F1EF0100F08BFB0ECD6
:1002D000108A80F30988BFF36F8F704718000020E1
:1002E000EFF3058070470000094880470948004740
:1002F000FEE7FEE7FEE7FEE7FEE7FEE7FEE7FEE7D6
:10030000FEE7FEE704480549054A064B7047000032
:10031000B52900088901000828300020283600206F
:10032000283200202832002053EA020C00F06980B5
:100330002DE9F04B4FF00006002B1FBFB3FA83F5F9
:1003400003FA05F424FA05F65E4012BF1643B2FA2A
:1003500082F502FA05F4C5F120051EBF22FA05FC5C
:1003600044EA0C04203556EA044C4FEA144418BF02
:10037000641C4FF000084FF00009904271EB030C31
:1003800039D3002919BFB1FA81F701FA07F6B0FA9B
:1003900080F700FA07F6C7F120071EBF20FA07FC16
:1003A00046EA0C062037B6FBF4FCA7EB0507103F26
:1003B00007F01F0BCBF120060CFA0BFB2CFA06F60C
:1003C00044BFB3460026202FA4BF5E464FF0000B6B
:1003D0005BEA060C08BF4FF0010B19EB0B09ABFBF6
:1003E000027C48EB0608C01B06FB02CC0BFB03CCCF
:1003F00071EB0C01C1E70B46024641464846BDE899
:10040000F08B13B54FF000004FF00001AFF3008008
:10041000BDE81C407047032A40F2308010F0030C06
:1004200000F0158011F8013BBCF1020F624498BF47
:1004300011F801CB00F8013B38BF11F8013BA2F1E4
:10044000040298BF00F801CB38BF00F8013B11F05F
:10045000030300F05780083AC0F0088051F8043BCD
:10046000083A51F804CBA0E80810F5E7121D5CBF6C
:1004700051F8043B40F8043BAFF30080D20724BF9F
:1004800011F8013B11F801CB48BF11F8012B24BF33
:1004900000F8013B00F801CB48BF00F8012B704782
:1004A00002F0FF0343EA032242EA024200F05EB890
:1004B0004FF0000200B5134694469646203922BFFD
:1004C000A0E80C50A0E80C50B1F12001BFF4F7AF48
:1004D000090728BFA0E80C5048BF0CC05DF804EB2A
:1004E000890028BF40F8042B08BF704748BF20F898
:1004F000022B11F0804F18BF00F8012B7047704796
:100500007047704710B5203AC0F00B80B1E8185022
:10051000203AA0E81850B1E81850A0E81850BFF4ED
:10052000F5AF5FEA027C24BFB1E81850A0E818508C
:1005300044BF18C918C0BDE810405FEA827C24BFE0
:1005400051F8043B40F8043B08BF7047D20728BF6E
:1005500031F8023B48BF11F8012B28BF20F8023BBD
:1005600048BF00F8012B70474FF000020429C0F08B
:10057000128010F0030C3FF49DAFCCF1040CBCF1E1
:10058000020F18BF00F8012BA8BF20F8022BA1EB27
:100590000C01FFF78FBF5FEAC17C24BF00F8012B7D
:1005A00000F8012B48BF00F8012B7047754600F09A
:1005B0002BF8AE4605006946534620F007008546F5
:1005C00018B020B5FFF79EFEBDE820404FF00006B2
:1005D0004FF000074FF000084FF0000B21F007012B
:1005E000AC46ACE8C009ACE8C009ACE8C009ACE86E
:1005F000C0098D46704710B50446AFF30080204611
:10060000BDE81040FFF709BE00487047C82F002022
:1006100001491820ABBEFEE726000200704700002B
:100620004FF47A71484300EE100A9FED031AF8EE7A
:10063000400A80EE810A70470024744BF8B500250B
:1006400004462846009500F067F8060019D01D4FB3
:100650004FF4004500222946384600F057FC01209F
:1006600000F02AFB4FF0FF3302226946304601F0CA
:1006700077F901222946384600F048FCBDF8000011
:1006800045BA092004EB400131F8021C24F810108F
:10069000401E0028F6DC00210B4A2580084600BFDA
:1006A00032F81030401C19440A28F9DB0A20B1FB4B
:1006B000F0F09082A08AFFF7B3FF84ED060A0020D5
:1006C000F8BD000000040048AC2F002010B520B198
:1006D000012805D0022808D105E04FF4005304E0BA
:1006E0004FF4804301E04FF400430A4821B101294F
:1006F00005D002290BD107E01946012201E0194675
:10070000002200F003FC02E0194600F0F7FB002095
:1007100010BD00000008004808B1002070470148E3
:1007200070470000CC000020FEE710B5044600F042
:10073000DBF82046BDE8104000F096B970B586B0F1
:1007400006460820049000200D460092029041F2D7
:1007500088340390304600F0B1F810F0FF0F0BD052
:100760003CB102232A466946304600F03FF8002893
:1007700000D0012006B070BD012002F06BFE641EA7
:10078000E8D1F6E7014800F0E4B900007C01002060
:10079000014800F0DEB9000048020020054A016867
:1007A00011441422B1FBF2F1890001640249C163D2
:1007B00070470000F8FFFDBF0000024030B590F820
:1007C00040500124AC40C56B6C60046863604368B2
:1007D000102B036803D099600068C26030BD9A6036
:1007E0000068C16030BD704772B6FEE7F0B590F8A2
:1007F00020500468A468012D05D0022D03D0416A61
:1008000041F4802157E014F0406F01D1E5004FD54D
:10081000C4F301640125A5401D608D684FF4C073C9
:100820009DB1CE6835434E6845EAC605066803EBC0
:100830000417F5514FF4C275076805EB04150E69EE
:100840007E51097D012905D009E00E88CD6845EA71
:100850004655EBE701684E5946F480764E511179C2
:10086000D579567941EA056195792D0445EA062541
:1008700029434FF4C676056806EB0416A951117892
:10088000D57841EA0561957852782D0445EA02222F
:1008900011434FF4C475026805EB0415515100680B
:1008A00003EB0411425842F0010242500020F0BD17
:1008B000416A41F4001141620120F0BD024600206E
:1008C00092F82010012901D002290CD111688A6800
:1008D000520100D501208A68120100D5401C8968A8
:1008E000C90000D5401C704770B5040003D094F8CF
:1008F000200010B104E0012070BD204600F082F815
:100900002068016841F00101016000F005FB054627
:10091000052604E000F000FB401B0A2811D82068DF
:100920004068C007F6D02068016821F0020101602C
:1009300000F0F2FA05460BE000F0EEFA401B0A2840
:1009400006D9606A40F40030606284F82060D2E723
:10095000206840688007EFD4207E01282068016865
:100960003DD021F080010160607E0128206801688F
:1009700038D021F040010160A07E01282068016884
:1009800033D021F020010160E07E01282068016859
:100990002ED041F010010160207F012820680168FD
:1009A00029D021F008010160607F012820680168DA
:1009B00024D021F004010160D4E902010843D4E904
:1009C0000412114308436168491E08432168C86145
:1009D00000206062012084F82000002070BD41F0FA
:1009E0008001C0E741F04001C5E741F02001CAE7BE
:1009F00021F01001CFE741F00801D4E741F00401F4
:100A0000D9E7000010B586B0044614216846FFF708
:100A10004FFD1349206888421FD11248C16941F037
:100A20000071C161C16901F000710591416941F432
:100A3000003141614069694600F4003005904FF48F
:100A4000C0500090022001900020029003200390EB
:100A500009200490C00600F041F906B010BD000066
:100A6000006400400010024070B5044690F8200079
:100A7000012804D0606A40F40020606218E002207F
:100A800084F820002068016821F00101016000F075
:100A900043FA05460EE000BF00F03EFA401B0A286C
:100AA00008D9606A40F400306062052084F82000B4
:100AB000012070BD20684068C007EDD1606270BD44
:100AC00010B540B190F821100022022905D0042170
:100AD000816380F82020012010BD01680B6823F09D
:100AE0000E030B6001680B6823F001030B6090F8A4
:100AF0004030C46B012101FA03F3636080F82110D8
:100B000080F82020002010BD10B590F8211000249E
:100B1000022903D004218163012418E001680A68D6
:100B200022F00E020A6001680A6822F001020A60DF
:100B300090F84020C36B012101FA02F25A6080F85C
:100B40002110002180F82010416B01B18847204618
:100B500010BDF0B4C16B0D6801680C68066C04220E
:100B600002FA06F32B420FD063070DD50B689B06E4
:100B700003D40B6823F004030B6090F840108A4004
:100B8000C16B4A60C16A1BE0022303FA06F72F42D9
:100B90004FF0000C4FF0010216D0A70714D50C68D7
:100BA000A40605D40C6824F00A040C6080F8212007
:100BB00090F840108B40C16B4B6080F820C0816A78
:100BC000002918D0F0BC08470823B3402B4212D0AC
:100BD000230710D50B6823F00E030B6090F840102C
:100BE000C36B02FA01F15960826380F8212080F81A
:100BF00020C0016BE4E7F0BC704770B5040021D061
:100C0000022084F821002268116843F6F0708143C5
:100C1000D4E901031843D4E903352B43184363692E
:100C20001843A3691843E36918430843106020463A
:100C3000FFF7B4FD0020A063012184F8211084F89F
:100C4000200070BD012070BD70B5044690F82000F2
:100C5000002501280CD0012084F8200094F82160A0
:100C60000020012E06D084F820000225284670BD01
:100C7000022070BD022684F82160A0632068066807
:100C800026F0010606602046FFF798FDE06A00287E
:100C90002068016802D041F00E0106E041F00A012F
:100CA00001602068016821F004010160206801688A
:100CB00041F001010160D9E770B5044600F02CF95C
:100CC0000546601C02D004480078044400F024F972
:100CD000401BA042FAD370BD080000202DE9F04F60
:100CE000DFF80092002301260325A9F1040B85B04B
:100CF0000F2709F1040AABF1040EEAE006FA03F447
:100D000022407CD091F804C00CF0030CBCF1010F20
:100D100002D0BCF1020F26D1D0F808C0CDF800C037
:100D20004FEA430C05FA0CF8CDF810C0DDF800C00E
:100D30002CEA080CCDF800C0D1F80C80DDF810C00A
:100D400008FA0CF8DDF800C048EA0C08C0F8088082
:100D5000D0F804C02CEA040C0C79C4F300149C40B5
:100D600044EA0C0444600C79E443A4070DD0D0F8A5
:100D70000CC04FEA430805FA08F42CEA040C8C680E
:100D800004FA08F444EA0C04C4600C7904F0030487
:100D9000022C19D1DC0800EB84040294246A4FEA87
:100DA000437C4FEADC6CCDF810C007FA0CFC24EA57
:100DB0000C04D1F81080DDF810C008FA0CF848EAED
:100DC0000408029CC4F8208004684FEA430805FA2E
:100DD00008FC24EA0C0491F804C00CF0030C0CFA93
:100DE00008FC4CEA040CC0F800C04C6814F4403F06
:100DF0006ED03D4CD4F818C04CF0010C00E067E018
:100E0000C4F818C0A46923F0030C04F00104009492
:100E1000364C64440294A4684FEA837C4FEA1C7801
:100E200007FA08FC24EA0C04B0F1904F06D0DFF872
:100E3000C0C0604505D14FF0010C12E04FF0000C2E
:100E40000FE0DFF8B0C0604502D14FF0020C08E0BF
:100E5000DFF8A4C0604502D14FF0030C01E04FF071
:100E6000050C0CFA08FC4CEA040C029CC4F808C0FF
:100E7000D9F80040CC46D1F8048094435FEAC828F2
:100E800000D51443CCF80040DAF80040D446D1F83D
:100E9000048094435FEA882800D51443CCF80040CE
:100EA000DBF80040DC46D1F8048094435FEA8838E0
:100EB00000D51443CCF80040DEF80040F446D1F8E9
:100EC000048094435FEAC83800D51443CCF800404E
:100ED0005B1C0A6832FA03F47FF410AF05B0BDE87A
:100EE000F08F0000080401400010024000000140A3
:100EF0000004004800080048000C0048426921EA4C
:100F000002030A4043EA0241816170470AB18161EC
:100F10007047816270470000014880687047000098
:100F200008000020024881680278114481607047FF
:100F300008000020074810B5016841F01001016069
:100F4000032000F071F80F2000F006F800F024F8FC
:100F5000002010BD0020024070B50D4D04464FF436
:100F60007A712878B1FBF0F00A490968B1FBF0F01A
:100F700000F0EBFE48B9102C07D200222146501E8B
:100F800000F032F800206C6070BD012070BD0000E0
:100F900008000020140000200B4882B0816941F055
:100FA00001018161816901F001010091C16941F094
:100FB0008051C161C069002200F0805000900F2173
:100FC000901E02B000F010B800100240002809DBAB
:100FD00000F01F02012191404009800000F1E02053
:100FE000C0F8001170470000F0B40E4B1B680C46AF
:100FF000C3F30223C3F10705042D00D90425191DED
:10100000072901D2002300E0DB1E012606FA05F1C4
:10101000491E214099409E40761E16403143F0BC47
:1010200002F0A5B90CED00E0064900F007020868DF
:101030004FF6FF03184040EA0220034A10430860BD
:10104000704700000CED00E00000FA052DE9F047C4
:101050000F46050069D04A4E306800F00700B842DC
:1010600009D2306820F0070038433060306800F063
:101070000700B84259D12878424C800705D56068EE
:10108000A96820F0F000084360602878C0073DD0D0
:101090006968012001290DD0022923D05FF00203E5
:1010A00093FAA3F2B2FA82F242F02002520904D07B
:1010B000226803E04FF40033F2E7626A93FAA3F385
:1010C000B3FA83F303F01F03984002422DD0606807
:1010D00020F0030008436060FFF71EFF804641F2E6
:1010E00088390CE04FF00073DAE700BFFFF714FF18
:1010F000A0EB0801494502D90320BDE8F0876068EC
:10110000696800F00C00B0EB810FEFD1306800F09F
:101110000700B8420BD9306820F007003843306030
:10112000306800F00700B84201D00120E5E72878D8
:10113000400705D56068E96820F4E0600843606016
:101140002878000706D56068296920F4605040EAD5
:10115000C100606000F04EF86168F02292FAA2F2DD
:1011600001F0F001B2FA82F2D140074A515CC84066
:101170000649086006480068FFF7EEFE0020BCE75D
:1011800000200240001002409C5100081400002082
:101190000C00002008480949006849684FF4E062E3
:1011A00092FAA2F201F4E061B2FA82F2D140044A6A
:1011B000515CC8407047000014000020001002403D
:1011C000AC51000808480949006849684FF460526A
:1011D00092FAA2F201F46051B2FA82F2D140044ACA
:1011E000515CC8407047000014000020001002400D
:1011F000AC5100080F4A10B551680F4801F00C03BC
:10120000042B12D0082B10D10C4BC1F38344D26AAB
:101210001C5D02F00F021033C9039A5C06D500234F
:101220001946FFF781F8A0FB040110BD0448A4FB98
:10123000000110BD0010024000127A007C5100082D
:1012400000093D002DE9F84F050071D02878FC4ECB
:10125000C0074FF0010425D070686704C0F3810017
:10126000012807D07068C0F3810002281BD1706884
:10127000C00318D597FAA7F0B0FA80F040F020002C
:10128000400901D0306800E0706A97FAA7F1B1FA1E
:1012900081F101F01F0104FA01F1084265D068688C
:1012A0000028D2D061E06868B0F5803F0BD010B163
:1012B000B0F5A02F17D0306820F48030306030684F
:1012C00020F4802002E0306840F480303060F06A22
:1012D000A96820F00F000843F062686820B3FFF7A8
:1012E0001BFE80460AE0306840F480203060EAE768
:1012F000FFF712FEA0EB0800642871D897FAA7F058
:10130000B0FA80F040F02000400901D0306800E0E1
:10131000706A97FAA7F1B1FA81F101F01F0104FA9E
:1013200001F10842E4D020E0FFF7F6FD804607E037
:10133000C2E000BFFFF7F0FDA0EB08006428DCD896
:1013400097FAA7F0B0FA80F040F02000400901D0F1
:10135000306800E0706A97FAA7F1B1FA81F101F004
:101360001F0104FA01F10842E4D12878DFF8D482A1
:1013700080074FF0000A4FF0020730D570684FF039
:10138000F80B10F00C0F07D07068C0F38100022832
:1013900027D17068C00324D497FAA7F0B0FA80F080
:1013A00040F02000400901D0306800E0706A97FAF0
:1013B000A7F1B1FA81F101F01F0104FA01F108422D
:1013C00002D02869012877D130689BFAABF220F06F
:1013D000F8016869B2FA82F29040014331605AE044
:1013E00064E1286988B394FAA4F0B0FA80F048F870
:1013F0002040FFF791FD814606E000BFFFF78CFD1E
:10140000A0EB090002289AD897FAA7F0B0FA80F06A
:1014100040F02000400901D0306800E0706A97FA7F
:10142000A7F1B1FA81F101F01F0104FA01F10842BC
:10143000E4D030689BFAABF26969B2FA82F220F02C
:10144000F80091400843306025E0FFE794FAA4F0EB
:10145000B0FA80F048F820A0FFF75EFD814605E075
:10146000FFF75AFDA0EB09000228CCD897FAA7F0A5
:10147000B0FA80F040F02000400901D0306800E070
:10148000706A97FAA7F1B1FA81F101F01F0104FA2D
:1014900001F10842E4D1287800076CD5A869A8B307
:1014A00094FAA4F0B0FA80F008EB8000C0F8804411
:1014B000FFF732FD814607E0A4E100BFFFF72CFDF6
:1014C000A0EB090002289ED897FAA7F0B0FA80F0A6
:1014D00040F06000B4EB501F01D130680BE097FA88
:1014E000A7F0B0FA80F040F06000B7EB501F01D1D8
:1014F000306A00E0706A97FAA7F1B1FA81F101F061
:101500001F0104FA01F21042D8D034E0FFE794FA48
:10151000A4F1B1FA81F108EB8101C1F880A4FFF7D1
:10152000FBFC814606E000BFFFF7F6FCA0EB0900DC
:1015300002289AD897FAA7F0B0FA80F040F060003D
:10154000B4EB501F01D130680BE097FAA7F0B0FA66
:1015500080F040F06000B7EB501F01D1306A00E02E
:10156000706A97FAA7F1B1FA81F101F01F0104FA4C
:1015700001F21042D8D12878400768D5F0694FF0C1
:101580000009C00009D4F06940F08050F061F069B2
:101590004FF0010900F0805000902B480168C90508
:1015A00012D4016841F480710160FFF7B5FC8346F5
:1015B00006E000BFFFF7B0FCA0EB0B00642875D875
:1015C00021480068C005F5D5E86801280AD008B1AF
:1015D000052811D0306A20F001003062306A20F016
:1015E000040002E0306A40F001003062E86868B34D
:1015F000FFF792FC83460DE0306A40F00400306251
:10160000F0E700BFFFF788FCA0EB0B0141F2883048
:1016100081424BD897FAA7F0B0FA80F040F0400032
:10162000B4EB501F01D1306813E097FAA7F0B0FA7D
:1016300080F040F04000B7EB501F09D1306A08E05D
:101640000010024000004242007000400CE040E008
:10165000706A97FAA7F1B1FA81F101F01F0104FA5B
:1016600001F21042CED02DE0FFF756FC834607E092
:10167000FFF752FCA0EB0B0141F28830814215D8F4
:1016800097FAA7F0B0FA80F040F04000B4EB501F9A
:1016900001D130680CE097FAA7F0B0FA80F040F082
:1016A0004000B7EB501F02D1306A01E083E0706A5E
:1016B00097FAA7F1B1FA81F101F01F0104FA01F2E2
:1016C0001042D5D1B9F1000F03D0F06920F080505D
:1016D000F061E86980B37168C1F38101022977D0B4
:1016E0004FF080714F000228504609D091FAA1F1C5
:1016F000B1FA81F148F82100FFF70EFC05465DE0E4
:10170000894691FAA1F1B1FA81F1C24648F8210067
:10171000FFF702FC804605E0FFF7FEFBA0EB0800A8
:10172000022848D897FAA7F0B0FA80F040F02000DD
:10173000400902D0306801E066E0706A97FAA7F1CC
:10174000B1FA81F101F01F0104FA01F10842E3D17D
:10175000D5E908100843716821F4741108437060DA
:1017600099FAA9F0B0FA80F04AF82040FFF7D4FBCC
:10177000054604E0FFF7D0FB401B02281BD897FA70
:10178000A7F0B0FA80F040F02000400901D03068A6
:1017900000E0706A97FAA7F1B1FA81F101F01F0138
:1017A00004FA01F10842E5D02EE000BFFFF7B4FBD8
:1017B000401B022802D90320BDE8F88F97FAA7F052
:1017C000B0FA80F040F02000400902D0306801E01B
:1017D0000BE0706A97FAA7F1B1FA81F101F01F01ED
:1017E00004FA01F10842E1D10EE00128E4D070686A
:1017F0002A6A00F48031914204D1696A00F47010C1
:10180000884201D00120D7E70020D5E770B5040059
:1018100009D0606A002540B125616561A56294F830
:101820005D0040B10CE0012070BD6068B0F5827FC2
:10183000F4D0E561F2E784F85C50204600F05CF8F3
:10184000022084F85D002068016821F040010160F9
:10185000E1684FF4E062914201D9002001E04FF4C9
:101860008050B1F5706F02D0914200D0A562A1887E
:10187000228901F4827102F404421143227C02F0B5
:1018800002021143227D02F001021143228B02F475
:1018900000721143227F02F03802114394F8202095
:1018A00002F080021143228D02F40052114322689B
:1018B0001160A169042202EA114194F8242000F485
:1018C000805002F01002114394F8342002F0080214
:1018D0001143A28902F47062114301432068416000
:1018E0002068C16921F40061C1612566012084F886
:1018F0005D00002070BD000010B586B004461421C4
:101900006846FEF7D5FD1349206888421FD112486A
:10191000C16941F48041C161C16901F4804105910F
:10192000416941F4802141614069694600F48020A9
:1019300005904FF4C04000900220019000200290DA
:1019400003200390052004900448FFF7C7F906B070
:1019500010BD0000003800400010024000040048A4
:101960002DE9F84F044690F85D00984616460F465C
:101970000025012801D00225ACE060684FF0040B7F
:10198000B0F5827F01D1A06830B394F85C000128E3
:101990002DD04FF0010984F85C90FFF7BDFA824624
:1019A000002F77D0002E75D084F85DB0002020661F
:1019B0002764A4F84460A4F84660A063A087E08789
:1019C000E0642065E0684FF4E06188422068426886
:1019D0000FD922F480520EE084F85DB013460A4617
:1019E0002046CDF8008000F07AF8BDE8F88F02209C
:1019F000FBE742F480524260A068B0F5004F09D185
:101A00002068026822F0400202602068026822F426
:101A10008042026020680268520603D4026842F0E5
:101A200040020260E06888421DD941E02068816878
:101A3000C9070BD0007B216C0870206C401C20640F
:101A4000B4F84600401EA4F846000CE0FFF764FA24
:101A5000A0EB0A01414503D3B8F1FF3F03D007E0F3
:101A6000B8F1000F04D0B4F846000028DED123E01E
:101A700003252DE020688168C9070CD0C068216C5F
:101A80000880206C801C2064B4F84600401EA4F836
:101A900046000DE01AE0FFF73FFAA0EB0A014145CE
:101AA00003D3B8F1FF3F03D0E2E7B8F1000FDFD076
:101AB000B4F846000028DDD152464146204600F0E9
:101AC0000DFE08B120202066206E08B1012501E03E
:101AD00084F85D90002084F85C00284685E72DE9B5
:101AE000FF5F044690F85C0000260E9F1D4693465B
:101AF0004FF0010901280FD04FF0010A84F85CA0D3
:101B0000FFF70AFA804694F85D00616801280DD05D
:101B1000B1F5827F08D103E0022004B0BDE8F09F58
:101B2000A16809B9042801D0022609E1019800281A
:101B300076D0BBF1000FFBD0002DF9D094F85D00FA
:101B4000042802D0052084F85D0000202066C4F837
:101B500040B0A4F84650A4F844500199A163E58729
:101B6000A587E0642065E0684FF4E061884201D811
:101B7000012D04D92068426822F4805203E02068D5
:101B8000426842F48052426020680268520603D4E0
:101B9000026842F040020260E0688842606848D90A
:101BA00008B1012D3DD1A06B21680088C860A06BF1
:101BB000801CA063E08F401EE08732E020688168CF
:101BC00089070FD5E18F69B1B9F1010F0AD1A16B76
:101BD0000988C160A06B801CA063E08F401EE08775
:101BE0004FF0000920688168C9070FD0B4F846108B
:101BF00061B1C068216C0880206C801C2064B4F83E
:101C00004600401EA4F846004FF00109FFF784F992
:101C1000A0EB0800B84204D3781C02D003268DE064
:101C20008AE0E08F0028C9D1B4F846000028C5D169
:101C300077E008B1012D6DD1E08F0128A06B08D9A4
:101C400021680088C860A06B801CA063E08F801EA4
:101C500007E0216800780873A06B401CA063E08F48
:101C6000401EE08756E02068816889071AD5E18F19
:101C7000C1B1B9F1010F15D1E18F0129A16B07D9CC
:101C80000988C160A06B801CA063E08F801E06E005
:101C900009780173A06B401CA063E08F401EE087B1
:101CA0004FF0000920688168C90728D0B4F84610B1
:101CB00029B3B4F84610012914D9C068216C0880F2
:101CC000206C801C2064B4F84600801EA4F84600F6
:101CD000B4F84600012810D82068416841F48051CA
:101CE00041600AE0007B216C0870206C401C20647D
:101CF000B4F84600401EA4F846004FF00109FFF773
:101D00000BF9A0EB0800B84202D3781C02D085E79B
:101D1000002F83D0E08F0028A5D1B4F8460000281A
:101D2000A1D142463946204600F012FD10B10126ED
:101D300020202066206E08B1012601E084F85DA015
:101D4000002084F85C003046E7E610B5401EB0F194
:101D5000807F01D3012010BD4FF0E02460610F218E
:101D6000601701F004FB0020A06107202061002023
:101D700010BD0000F0B590F83C20012A29D00124C4
:101D800080F83C40022280F83D2003685A689D6834
:101D9000114EB34203D122F470074A683A4322F04D
:101DA00070070A683A435A600268B24205D0B2F13D
:101DB000804F02D0094B9A4204D1896825F08003F4
:101DC0001943916080F83D40002180F83C1008469E
:101DD000F0BD0220F0BD0000002C01400040014099
:101DE00010B586B0044614216846FEF761FB2068F2
:101DF000B0F1804F17D10D48416941F40031416184
:101E00004069694600F400300590042000900220EB
:101E100001900020029003200390012004904FF0D5
:101E20009040FEF75BFF06B010BD000000100240BE
:101E300070B5044690F83C0000260D4601280BD0F2
:101E4000012084F83C000C2A4AD007DC82B1042A25
:101E500020D0082A06D131E0022070BD102A53D0CC
:101E6000142A63D00126002084F83C00304670BD5F
:101E7000206800F0EBFD2068816941F00801816174
:101E80002068816921F004018161206881692A69E3
:101E9000114311E0206800F01DFE2068816941F4C3
:101EA000006181612068816921F48061816120681D
:101EB00081692A6941EA02218161D4E7206800F042
:101EC00049FE2068C16941F00801C1612068C1690B
:101ED00021F00401C1612068C1692A69114311E040
:101EE000206800F077FE2068C16941F40061C1619B
:101EF0002068C16921F48061C1612068C1692A69D3
:101F000041EA0221C161AEE7206800F099FE206835
:101F1000416D41F0080141652068416D21F00401E7
:101F200041652068416D2A69114311E0206800F085
:101F3000B9FE2068416D41F4006141652068416D42
:101F400021F4806141652068416D2A6941EA0221DE
:101F5000416588E710B5040003D094F83D0010B146
:101F600007E0012010BD002084F83C00204600F06E
:101F700023F8022084F83D00211D206800F022FD96
:101F8000012084F8480084F83E0084F83F0084F87B
:101F9000400084F8410084F8420084F8430084F84B
:101FA000440084F8450084F8460084F8470084F82B
:101FB0003D00002010BD000038B505460068B0F1B6
:101FC000804F20D11048C16941F00101C161C06951
:101FD0000F4C00F0010000900C4820601020606061
:101FE00000208021C4E9020189002161890061612A
:101FF0002021C4E906102046FEF7FFFD08B1FEF7D8
:10200000F3FBEC62656238BD00100240080002403C
:102010007C01002070477047704700002DE9F041B7
:1020200002680446D0691168936840F60F0528429B
:102030004FF000054FF0020605D187067ED58F06CA
:102040007CD5A16E2AE1DFF884C203F0010701EA22
:102050000C0C57EA0C0C71D05FEAC07C0CD05FEA24
:10206000C15C09D54FF0010CC2F820C0D4F884201F
:1020700042F00102C4F88420820709D5DA0707D0AC
:1020800022681662D4F8842042F00402C4F8842046
:1020900042070AD5DA0708D0236804221A62D4F866
:1020A000842042F00202C4F8842002070CD501F01B
:1020B00020023A4308D0236808221A62D4F8842008
:1020C00042F00802C4F8842002050BD54A0109D564
:1020D00023684FF400621A62D4F8842042F0200290
:1020E000C4F88420D4F88420002A36D0800605D590
:1020F000880603D5A16E09B120468847D4F884002C
:1021000021688968490602D410F0280F27D020469C
:1021100001F00AF82068806840061BD52068083066
:1021200050E8001F21F0400140E80012002AF5D1DC
:10213000606F78B166494163606F00E015E0FEF7BB
:10214000E3FC002809D0606F416B00E02046BDE849
:10215000F04108472046FFF75FFFBDE8F0812046C9
:10216000FFF75AFFC4F88450F7E7D4F860C020277F
:10217000BCF1010F7DD15FEAC06C7ED55FEAC16C16
:102180007BD51020106220688068400642D5616FC0
:10219000086840680004000CDFD0B4F85820824280
:1021A000DBD9A4F85A00886920282BD0216851E88F
:1021B000000F20F4807041E80002002AF6D1206868
:1021C000083050E8001F21F0010140E80012002A09
:1021D000F5D12068083050E8001F21F0400140E8A8
:1021E0000012002AF5D1C4F880702566206850E8F6
:1021F000001F21F0100140E80012002AF6D1606FA4
:10220000FEF75EFC6666B4F85800B4F85A10401A3F
:1022100081B22CE0B4F85800B4F85A10401A81B2D8
:10222000B4F85A00002898D0002996D0226852E8C5
:10223000000F20F4907042E80003002BF6D12068D4
:10224000083050E8002F22F0010240E80023002B64
:10225000F5D1C4F880702566A566206850E8002F87
:1022600022F0100240E80023002BF6D166662046DB
:1022700000E002E0FFF7CEFE6FE7C60209D55B0281
:1022800007D54FF4801010622046BDE8F041FFF7FB
:10229000C2BE020606D50A0604D5E16E00297FF407
:1022A00055AF5AE74006E7D54806E5D5204602680F
:1022B00052E8001F21F0400142E80013002BF6D144
:1022C000C767C56600F0D4F847E7000020010004A6
:1022D0007D30000810B5040002D0E06F10B107E0B7
:1022E000012010BD002084F87800204600F026F878
:1022F0002420E0672068016821F001010160606A24
:1023000010B1204600F002FE204600F03FFF0128F9
:10231000E7D02068416821F49041416020688168DD
:1023200021F02A0181602068016841F0010101600B
:102330002046BDE8104000F04DBE000070B586B0EC
:10234000064614216846FEF7B3F8214930688842F2
:102350003BD12049C86940F48020C861C86900F4B5
:1023600080200590486940F4802048614869002534
:1023700000F4802005904FF4406000900220CDE9E9
:102380000105032003900720049069461248FEF7D8
:10239000A5FC134C114820601020C4E901058020E1
:1023A000C4E903056561A5612046E561FEF725FCEA
:1023B00008B1FEF719FA346700220521272066626A
:1023C000FEF712FE2720FEF701FE06B070BD0000EA
:1023D0000048004000100240000400481C00024079
:1023E0004802002070B50446C06F202801D00220AA
:1023F00070BD29B322B3E164A4F85020A4F85220A0
:102400000021C4F884102120E067206FD0B1154B63
:102410008362236F1448D862236F14481863206FB7
:10242000134641632068256F00F128022846E16CBD
:10243000FEF70AFC30B11020C4F884002020E067C9
:10244000012070BD2168402008622068083050E8F3
:10245000001F41F0800140E80012002AF5D1002061
:1024600070BD0000DF3000081F3100089130000807
:1024700070477047FEE700000F4810B50D49016036
:102480000421416000214FF440328160C0E9031211
:1024900012014261017641768176C17601774177FA
:1024A000FEF722FA002803D0BDE81040FEF79CB9E1
:1024B00010BD000000640040A40000200D4808B5D5
:1024C000416941F0010141614069002200F00100D1
:1024D000009005210B20FEF787FD0B20FEF776FD0F
:1024E000002205210C20FEF77FFDBDE808400C20EE
:1024F000FEF76CBD0010024010B5074A00210748E6
:1025000001F06AF9064C074A00216060064801F0B4
:1025100063F9206010BD00005851000831290008FF
:1025200000000020B4510008E52D0008F0B587B088
:1025300014216846FDF7BCFF2448416941F400219D
:102540004161416901F400210591416941F4800133
:102550004161416901F480010591416941F4003113
:102560004161416901F400310591416941F48021E3
:1025700041614069164E00F480204FF4604405909C
:10258000002221463046FEF7C1FC124F0122110302
:102590003846FEF7BBFC002279013846FEF7B6FC50
:1025A0000125CDE900450024029469463046039494
:1025B000FEF794FBF0130090CDE9015469463846CC
:1025C0000394FEF78BFB07B0F0BD00000010024043
:1025D0000008004800040048134810B51149016084
:1025E0004FF4827141604FF4806181604FF4E0618B
:1025F000C16000214FF400720161C0E90512082298
:10260000C0E9072107234162C0E90A13C0E90C129F
:10261000FFF7FCF8002803D0BDE81040FEF7E4B84F
:1026200010BD000000380040CC00002010B58AB07A
:102630000024079408941C2168460994FDF738FF8C
:1026400015484FF08041C0E900145921C0E902410A
:1026500004618461FFF77EFC08B1FEF7C5F80794BA
:1026600007A90D480994FFF785FB08B1FEF7BCF8F0
:102670006020CDE9000404200490082269460294F9
:102680000548FFF7D5FB08B1FEF7AEF80248FFF7A3
:10269000A7FB0AB010BD0000300100200D4810B5A6
:1026A0000B4901604FF4E1314160002181600C224F
:1026B000C160C0E904128161C16101624162FFF73A
:1026C00009FE002803D0BDE81040FEF78DB810BD0C
:1026D00000480040C0010020FEE7FEE72DE9F84376
:1026E000044640684FF48276154689464FF4004709
:1026F0004FF48068B04209D1A068B84201D040458B
:1027000004D12068016821F0400101604B4600229D
:1027100080212046009500F0AFF880B96068B04293
:1027200014D1A068B84201D040450FD14B460022D9
:102730004FF4C0612046009500F02EF830B1206EB5
:1027400040F0200020660320BDE8F8830020FBE76E
:10275000F8B515460E460B460092044600224FF48B
:10276000C05100F019F888B9334600228021204674
:10277000009500F081F848B9334600224FF4C0615B
:102780002046009500F008F8002804D0206E40F0A4
:10279000200020660320F8BD2DE9FE4F4FF0000A0F
:1027A000984617460E4604460C9D8DF804A0FEF789
:1027B000B3FB411BA8EB0105FEF7AEFB8146206889
:1027C0004FF4C06B0C3002902A480068C0EBC00088
:1027D00000EB8000000D6843009043E05E4506D1A9
:1027E0002FB9029800788DF804009DF80400B8F124
:1027F000FF3F37D0FEF790FBA0EB0900A84203D2C1
:1028000015B1009858B32BE02068416821F0E00131
:1028100041606068B0F5827F0BD1A068B0F5004FD1
:1028200002D0B0F5806F04D12068016821F040012A
:102830000160A06AB0F5005F09D12068016821F449
:10284000005101602068016841F4005101600120DD
:1028500084F85D0084F85CA00320BDE8FE8F0025AD
:10286000401E0090206880683040B842B6D10020F9
:10287000F3E70000140000202DE9F8431E469146BE
:1028800088460446089DFEF747FB401B351AFEF7B5
:1028900043FB074625480068C0F3CB30684338E067
:1028A000701C37D0FEF738FBC01BA84203D215B10D
:1028B000009860B32CE02068416821F0E00141609D
:1028C0006068B0F5827F0BD1A068B0F5004F02D0F0
:1028D000B0F5806F04D12068016821F040010160EB
:1028E000A06AB0F5005F09D12068016821F40051A9
:1028F00001602068016841F400510160012084F802
:102900005D00002084F85C000320BDE8F88300250A
:10291000401E00902068816838EA010004D0002140
:102920004945BDD10020F0E70121F9E7140000205E
:1029300010B500F03DFFBDE8104000F09FBF10B59E
:10294000FEF7F0FA02F044FA012803D0BDE8104087
:1029500001F0FCBE10BD30B58FB028216846FDF7F0
:10296000A7FD14210AA8FDF7A3FD01210804CDE964
:1029700000100024029402250491CDE907504FF481
:10298000E01009906846FEF75DFC08B172B6FEE7FC
:102990000F20CDE90A054FF48060CDE90C400221FB
:1029A0000AA80E94FEF752FB002801D072B6FEE78B
:1029B0000FB030BD0248016841F4700101607047FA
:1029C00088ED00E0F0B502681C4B4FF0804798425C
:1029D00001D0B84203D122F070044A682243184C57
:1029E000184D194E984207D0B84205D0A04203D0E6
:1029F000A84201D0B04203D122F44077CA683A43DA
:102A00004F6922F080023A4302608A68C2620A6813
:102A10008262984205D0A04203D0A84201D0B042C1
:102A200001D109690163012141610169C90703D02D
:102A3000016921F001010161F0BD0000002C01409D
:102A4000004001400044014000480140F0B5056AE3
:102A5000026A22F00102026243688269184C25F082
:102A6000020522400C6822F0030214438A68164EC5
:102A70002A43144D154FDFF858C0A84205D0B04284
:102A800003D0B84201D0604506D122F0080ECA68D2
:102A900042EA0E0222F00402A84205D0B04203D05E
:102AA000B84201D0604505D14D6923F440731D4300
:102AB0008B692B4343608461496841630262F0BDC6
:102AC0008FFFFEFF002C0140004001400044014008
:102AD0000048014030B5046A026A22F01002026226
:102AE00042688369164D2B400D6823F4407343EA16
:102AF000052524F020038C6843EA0413114CA042FE
:102B000007D1CC6823F0800343EA041323F0400389
:102B100008E00D4CA04205D00C4CA04202D00C4C59
:102B2000A04207D14C6922F4406242EA84028C69D7
:102B300042EA84024260856149688163036230BD74
:102B4000FF8FFFFE002C0140004001400044014087
:102B50000048014030B5046A026A22F480720262C1
:102B60004268C369164D2B400D6823F003031D43D3
:102B700024F400738C6843EA0423124CA04207D16A
:102B8000CC6823F4006343EA042323F4806308E061
:102B90000D4CA04205D00D4CA04202D00C4CA042DE
:102BA00007D14C6922F4405242EA04128C6942EA8D
:102BB00004124260C5614968C163036230BD000010
:102BC0008FFFFEFF002C0140004001400044014007
:102BD0000048014030B5046A026A22F48052026261
:102BE0004268C369114D24F400542B400D6823F44E
:102BF000407343EA05238D6844EA05340C4DA8422E
:102C000008D00C4DA84205D00B4DA84202D00B4D68
:102C1000A84204D14D6922F4804242EA8512426002
:102C2000C36149680164046230BD0000FF8FFFFE8C
:102C3000002C014000400140004401400048014098
:102C400030B5046A026A22F4803202624268436D3F
:102C50000F4D2B400D681D4324F400330C8943EACB
:102C600004430C4CA04208D00B4CA04205D00B4CA6
:102C7000A04202D00A4CA04204D14C6922F4803216
:102C800042EA04224260456549688165036230BDBD
:102C90008FFFFEFF002C0140004001400044014036
:102CA0000048014030B5046A026A22F480120262D0
:102CB0004268436D104D24F400142B400D6843EA24
:102CC00005230D8944EA05540C4DA84208D00C4D4B
:102CD000A84205D00B4DA84202D00B4DA84204D10A
:102CE0004D6922F4802242EA8522426043654968A8
:102CF000C165046230BD0000FF8FFFFE002C014063
:102D000000400140004401400048014000F0EEFB5B
:102D1000C821B0FBF1F700F0D5FB0646104800F0E3
:102D200037FB0F4C0F4D04F1140818343E440C4887
:102D3000FDF784FC686900F01DFD00231A4641463A
:102D4000686900F0D7FCA86900F014FD00231A465A
:102D50002146A86900F0CEFC304600F095FBE5E77F
:102D6000AC2F0020602F002008B500F0BFFB6421CD
:102D7000B0FBF1F600F0A6FB05461748FDF7D5FCC1
:102D80000020164F164CADF800004FF00A083544ED
:102D9000642300226946786900F034FC68B9BDF804
:102DA0000000010A2170607022890D490A48FDF770
:102DB000C5FCA072E068401CE060E168B1FBF8F27D
:102DC00008FB121018B902210120FDF77FFC2846EC
:102DD00000F05AFBDBE70000A4000020602F002079
:102DE0009000002010B500F0A1FB194A00211948FD
:102DF00000F0F2FC184C194A00216060184800F0FD
:102E0000EBFC2060174A0021174800F0E5FCE06069
:102E1000164A0021164800F0DFFCA06000220821BD
:102E2000022000F02DFC606100220821022000F049
:102E300027FC206100220421022000F021FCA06177
:102E400000F0B6FB00F0B4FCBDE8104000F016BD89
:102E5000FC5100080D2D0008602F0020D8510008FB
:102E6000692D000820520008752E00084452000801
:102E7000C92E000800F03AFB064600F023FBDFF8FD
:102E80003C800F4F05460024354402210020FDF709
:102E90001DFCF868A0420BD1D8F8000000F0EEFC51
:102EA00000221146074800F097FCC8F8000000E037
:102EB0000446284600F0E8FAE6E70000602F00200C
:102EC00090000020692D000800F010FB3221B0FBBB
:102ED000F1F500F0F7FA0A4E04464FF0FF372C44A4
:102EE0003B4600220749B06900F08CFB20B9042260
:102EF00004490548FFF776FA204600F0C5FAEEE7E8
:102F0000602F0020A0000020C001002090F82410B5
:102F1000090706D501684A68436B22F400421A4348
:102F20004A6090F82410C90706D001684A68836A8D
:102F300022F400321A434A6090F82410890706D51B
:102F400001684A68C36A22F480321A434A6090F8E2
:102F50002410490706D501684A68036B22F48022D1
:102F60001A434A6090F82410C90606D501688A6899
:102F7000836B22F480521A438A6090F824108906E9
:102F800006D501688A68C36B22F400521A438A602E
:102F900090F82410490611D501684A68036C22F4A0
:102FA00080121A434A60016CB1F5801F06D1016896
:102FB0004A68436C22F4C0021A434A6090F8241015
:102FC000090606D501684A68806C22F40022024393
:102FD0004A6070472DE9F84300260446C0F8846033
:102FE000FDF79AFF8046206800684FF02005000733
:102FF0006FF07E4712D543460022290420460097F1
:1030000000F064F950B1216851E8000F20F0800011
:1030100041E80002002AF6D1E56721E02068006857
:10302000400722D5434600224FF4800120460097F6
:1030300000F04CF9C8B1216851E8000F20F49070FD
:1030400041E80002002AF6D12068083050E8001F4D
:1030500021F0010140E80012002AF5D1C4F88050A7
:1030600084F878600320BDE8F883E567C4F88050F1
:1030700044F8606F666026760020F4E710B5406A79
:103080000021A0F85A10A0F85210FEF7C5FF10BD9D
:1030900070B5446AE06FD4F88050216889684FF0B9
:1030A0000006090606D5212804D1A4F8526020465E
:1030B00000F060F820688068400606D5222D04D113
:1030C000A4F85A60204600F02FF8D4F8840040F0AD
:1030D0001000C4F884002046FEF79EFF70BD10B5B6
:1030E0000146406A8969202916D00021A0F85210B3
:1030F0000168083151E8002F22F0800241E80023E6
:10310000002BF5D1026852E8001F41F0400142E86F
:103110000013002BF6D110BDFFF7AAF910BD10B5B2
:10312000406AFFF7A6F910BD016851E8002F22F4AC
:10313000907241E80023002BF6D10168083151E874
:10314000002F22F0010241E80023002BF5D1016E8F
:10315000012908D1026852E8001F21F0100142E85D
:103160000013002BF6D12021C0F880100021016649
:1031700081667047026852E8001F21F0C00142E8F2
:103180000013002BF6D12021C167704770B50446AB
:1031900080682169E269084361690025114322685A
:1031A00008431168434B194001431160206841688E
:1031B000E26821F4405111434160A169206A08434B
:1031C00021688A6822F4306202438A603A492068A2
:1031D000884210D13948006B10F0030011D001284B
:1031E00005D0022805D003280DD102210CE00421CE
:1031F0000AE0082108E03249884202D03149884279
:1032000001D1002100E01021E3694FF400402E4A73
:103210004FF6EF76834226D1092941D2DFE801F04B
:1032200005080B400D4040401000FDF7B3FF06E0DD
:10323000FDF7C8FF03E0104602E0FDF7DBFF80B3B7
:103240004100606801EB5001B1FBF0F0A0F110010A
:10325000B14225D84FF6F0710140C0F3420001435E
:103260002068C16021E009291AD2DFE801F00508D1
:103270000B190D1919191000FDF78CFF06E0FDF769
:10328000A1FF03E0104602E0FDF7B4FF48B161681A
:1032900000EB5100B0FBF1F0A0F11001B14201D9F7
:1032A000012502E0216880B2C8600020A066E066C7
:1032B000284670BDF369FFEF00380140001002405E
:1032C000004400400048004000127A002DE9F04719
:1032D000994617460D4604464FF00008089E33E015
:1032E000701C31D0FDF718FEA0EB0900B04218D8D1
:1032F000BEB120680168490726D5802D24D0402D15
:1033000022D0C169C94309070DD4082505622046AA
:10331000FFF70AFFC4F8845084F878800120BDE8E4
:10332000F0870320FBE7C069C04300050CD4216887
:103330004FF4006008622046FFF7F6FE2020C4F834
:10334000840084F87880ECE72068C06935EA0000E2
:1033500004D00020B842C3D00020E0E70120F9E704
:103360000148FEF75BBE0000C0010020FEE7090730
:10337000090E002804DB00F1E02080F800147047FB
:1033800000F00F0000F1E02080F8141D70470000ED
:1033900070B5094C0546012211032046FDF7B6FD24
:1033A000002261012046FDF7B1FD1C212846FDF7F2
:1033B0007FF8002070BD00000004004870B50400D4
:1033C00005D0164E3068844209D1002070BD5020CF
:1033D00080F31188BFF34F8FBFF36F8FFEE700F0CC
:1033E000F3FE656900F010FF7068854202D0B06896
:1033F000854201D1022070BD0948854204D1A06AEE
:103400000028F7D1032070BD05481438854202D04A
:103410000DB1012070BD042070BD00001800002017
:103420007C070020FDF786FDFFF795FAFFF77EF891
:10343000FFF744F8FFF7D0F8FFF71EF8FFF7F6F8AC
:10344000FFF72CF900F056F8FFF756F800F090F867
:10345000FEE7000010B5EFF3058149B9EFF31081E5
:1034600031B908490968022905D1EFF3118111B179
:103470006FF0050403E0002408B100F079FF204656
:1034800010BD00006800002038B50546EFF3058048
:1034900048B9EFF3108030B909480068022805D117
:1034A000EFF3118010B16FF0050407E0002401F084
:1034B0009DFC291A0090684600F080FF204638BD28
:1034C00068000020EFF3058048B9EFF3108030B9B1
:1034D00005480068022804D1EFF3118008B101F01B
:1034E0008BBC01F083BC0000680000204FF47A70B0
:1034F00070470000EFF3058058B9EFF3108040B932
:1035000009490868022801D030B109E0EFF31180C1
:1035100030B16FF00500704701200860002070474F
:103520004FF0FF30704700006800002010B5EFF347
:10353000058048B9EFF3108030B90C4800680228C4
:1035400005D1EFF3118010B16FF0050010BD01F04F
:103550003FFC20B1022804D04FF0FF3010BD012005
:1035600010BD01F03FF8002010BD000068000020F1
:1035700010B5EFF3058060B9EFF3108048B90B493F
:103580000868022802D0012806D00BE0EFF3118072
:1035900040B16FF0050010BD0220086000F0DEFFB2
:1035A000002010BD4FF0FF3010BD0000680000206B
:1035B00070B5EFF3058048B9EFF3108030B91048CB
:1035C0000068022805D1EFF3118010B16FF00504F7
:1035D00013E001F0FDFB4FF0FF3510B102280BD1D5
:1035E00008E0012401F0ECFC012806D001F0F0FB1A
:1035F00010B102E0002400E02C46204670BD00001F
:1036000068000020F8B51D466FF003026FF0020657
:103610004FF00004EFF305834BB9EFF3108333B998
:10362000154B1B68022B17D1EFF31183A3B1F0B137
:10363000E9B1E5B9002200926A4601F0E3FA0128F7
:1036400017D10098B0B10D494FF080500860BFF31A
:103650004F8FBFF36F8F0DE048B141B12A4601F0A3
:1036600035FA012806D025B16FF0010402E01446B6
:1036700000E034462046F8BD6800002004ED00E07C
:10368000F8B514464FF00005EFF305826ABBEFF37F
:10369000108252BB164A1268022A02D1EFF311823D
:1036A0001ABB10B309B3ACB1D4E902326BB1502AE2
:1036B0001BD32269CAB1676900FB01F6B74214D374
:1036C0000025009501F07CF807E072B9226962B923
:1036D000626952B9002201F04FF8050005D00CB123
:1036E000216800E0002100F00DFE2846F8BD000032
:1036F00068000020F8B51D466FF003026FF0020667
:103700004FF00004EFF305834BB9EFF3108333B9A7
:10371000164B1B68022B18D1EFF31183ABB100B32A
:10372000F9B1F5B90022134600926A4601F070F92A
:10373000012818D10098B8B10D494FF080500860A9
:10374000BFF34F8FBFF36F8F0EE050B149B100232D
:103750002A4601F0ADF8012806D025B16FF001042A
:1037600002E0144600E034462046F8BD6800002020
:1037700004ED00E010B5EFF3058149B9EFF31081D6
:1037800031B90A490968022905D1EFF3118111B154
:103790006FF0050404E028B10024214601F044F84C
:1037A000204610BD6FF00304FAE700006800002017
:1037B000EFF3058048B9EFF3108030B90548006891
:1037C000022804D1EFF3118008B10020704701F006
:1037D000F9BA000068000020F0B585B04FEA010397
:1037E0004FF00004EFF305810394A1BBEFF31081C8
:1037F00089BB21490968022902D1EFF3118151BB2C
:1038000048B3802618218DF8104004AD42B31768E4
:1038100007B13D4697691FB139467F1E382F02D246
:103820001779FF0702D0002005B0F0BD576907B136
:10383000BE08D2F808C0BCF1000F0DD0D4685C2CD3
:1038400018D312693AB137B18DE8061032462946CD
:1038500001F08DFA03900DE0D7685FB912694AB99B
:1038600003AACDE90012B2B2294601F053FA0128A9
:1038700000D003940398D7E76800002070B5054690
:10388000EFF3058048B9EFF3108030B90D480068B8
:10389000022805D1EFF3118010B16FF005040FE09D
:1038A0004DB12846FFF78AFD042807D0002428469A
:1038B00000F0CAFD04E06FF0030401E06FF00204C1
:1038C000204670BD680000202DE9F041134C0F46E2
:1038D000054666692068001D00F01AFC681C07D1C7
:1038E00037B12168BDE8F0410D48091D00F060BC0A
:1038F00020683544B5424560216805D2A068BDE81E
:10390000F041091D00F03CBC6068091D00F038FC66
:10391000206B854200D22563BDE8F08118000020AD
:103920007C0700202DE9F041054600F04DFC2D4CB0
:103930002069401C206120682B4F10B1E06930B332
:103940002BE025602069012827D1002606EB8600A0
:1039500007EB800000F006FC761C382EF6D32348D7
:1039600000F000FC2148143000F0FCFB1F48283018
:1039700000F0F8FB1D483C3000F0F4FB1B485030D1
:1039800000F0F0FB194860601430A06005E020688A
:10399000E96AC06A884200D82560E06A401CE0629B
:1039A0006864E86AA169884200D9A06100EB8000E0
:1039B00007EB8000291D00F0FBFB00F025FCE0690F
:1039C00000280CD02068E96AC06A884207D20849FA
:1039D0004FF080500860BFF34F8FBFF36F8FBDE88B
:1039E000F081000018000020CC0200202C070020ED
:1039F00004ED00E038B500F0E7FB104CA068C8B952
:103A00000F4800F0AFFB0E48143000F0ABFB0C4841
:103A10002060143060600A4B00202833009003F1CE
:103A2000500210210A2000F0CBFEA06010B105A1C9
:103A300000F068FCBDE8384000F0E6BB5400002010
:103A400090070020546D72510000000030B4026CE9
:103A50000B46002A0BD0C1681144C1604468A142E2
:103A600001D30168C16030BC1846FCF7D4BC30BC3F
:103A700070472DE9F041856B174604460026026C1D
:103A800082B1C7B1E068FCF7C6FCE168206C091A96
:103A9000E1602268914202D26168081AE060022F58
:103AA00016D017E02068A8B9606801F011FA064640
:103AB000002060600EE0A068FCF7ADFC216CA068FF
:103AC0000844A0606168884204D32068A06001E0D7
:103AD00005B16D1E6D1CA5633046BDE8F08110B5C3
:103AE000044690F8590058B101280CD002280FD094
:103AF000502080F31188BFF34F8FBFF36F8FFEE725
:103B0000206B00F095FB2046BDE8104000F090BB14
:103B100010BD000010484FF40051420706D0C01DF0
:103B20000D4920F00700411AC1F500510B4A00234E
:103B30000144C2E900030839103A21F0070111607D
:103B40004B600B600B1AC0E9001393604FF000400C
:103B50005360D06070470000600F00207C000020A0
:103B6000144E154CA6F29C474FF08058DFF84C904D
:103B700012E000BF00F028FBF068C568281D00F0C7
:103B8000C7FA2069401E2061E068401EE06000F036
:103B90003BFB2846FFF7A3FFE0680028EAD138681E
:103BA0000128F9D9C9F80080BFF34F8FBFF36F8F99
:103BB000F2E70000680700201800002004ED00E094
:103BC00070B51D46049C51B1C4F80020C4E90F0132
:103BD0000121204600F028FE84F84C5070BD24607E
:103BE000F4E72DE9F0470E46DDE9098417468246E1
:103BF00091009946089DA522206BFCF751FC6FF0BF
:103C00000301206B01EB8701084420F007077807C8
:103C100007D0502080F31188BFF34F8FBFF36F8F11
:103C2000FEE72218315C82F83410315C11B1401C7F
:103C30001028F6D3002684F84360382D00D33725AA
:103C4000E562C4E91356201D00F097FA04F118004C
:103C500000F093FA2461C5F138006462A0616665E2
:103C600084F858604A465146384600F03BFA2060D6
:103C7000B8F1000F01D0C8F80040BDE8F08700009F
:103C800030B5114900E011460A688242FBD34B6807
:103C90005C18844203D14068184448600846436871
:103CA0001C18944209D1084C103C2468A24209D047
:103CB00052681A4442600A6812680260814200D069
:103CC000086030BD0460F9E77C00002070B5002476
:103CD00041600B4D0061914206D8D11A8269914230
:103CE00006D2011D686807E09A4203D2994201D3C7
:103CF000012403E0011D286800F042FA204670BD4F
:103D00005400002010B5044600F05EFAA06B28B104
:103D10005FF0000400F078FA204610BD0124F9E7B6
:103D200030B589B0304D55E00498002806DADDE959
:103D30000601059A9047049800284BDB069C6069B1
:103D400010B1201D00F0E4F902A800F0B9F8024615
:103D500004980A283ED2DFE800F00505053D263725
:103D600005053D260598A169034601442046FFF755
:103D7000ADFF00B3616A20468847E069012829D178
:103D8000002000900598A16900234218194620469A
:103D900001F0A8F978B9502080F31188BFF34F8F54
:103DA000BFF36F8FFEE70598A06128B18118134615
:103DB0002046FFF78BFF0DE0502080F31188BFF302
:103DC0004F8FBFF36F8FFEE794F82C0010B9204699
:103DD00000F02EFA002204A9A86800F077FE00285F
:103DE000A2D109B030BD0000540000202DE9FC41F3
:103DF0000F46054600F0F6FB01A800F061F8044606
:103E0000019818B101F0DCF8BDE8FC81224EAFB199
:103E100070680068A8B30027291B3A46B06800F014
:103E200085FA01F0CDF80028EED11C494FF0805002
:103E30000860BFF34F8FBFF36F8FE5E7A542EBD864
:103E400001F0BEF830682746C068C468201D00F045
:103E50005FF9E069012810D1A0692B4641193A4663
:103E60002046FFF733FF40B1002003460146009093
:103E70002A46204601F036F920B1616A204688477B
:103E8000C2E707E0502080F31188BFF34F8FBFF3E4
:103E90006F8FFEE70127BFE75400002004ED00E02C
:103EA00006484168096829B14168C968C968496814
:103EB000016370474FF0FF31FAE70000180000205F
:103EC00070B5054600F092FF064E04463069844204
:103ED00003D200F009F8012000E00020286020460D
:103EE000346170BD54000020F8B5194D1FE0C06862
:103EF000C4680668201D00F00BF9616A20468847F7
:103F0000E069012813D1A0693044B04206D9246188
:103F10006060211D286800F033F908E000200346A6
:103F2000014600903246204601F0DCF838B128689E
:103F300001680029DBD16968C5E90010F8BD50208F
:103F400080F31188BFF34F8FBFF36F8FFEE7000040
:103F50005400002008484068401C4FF0500080F397
:103F6000118804D0BFF34F8FBFF36F8FFEE7BFF30D
:103F70004F8FBFF36F8FFEE784000020074C20684F
:103F8000016841B1C0680021D0F80000FFF72EFFA2
:103F9000FFF7C6FEF3E701210020F7E754000020F9
:103FA0002DE9F041044600F00FF994F9455004F171
:103FB000240609E0606A48B1304600F0C9FF08B144
:103FC00000F092FA6D1E6DB2002DF3DC4FF0FF365B
:103FD00084F8456000F018F900F0F6F894F94450C0
:103FE00004F1100709E0206948B1384600F0B0FF3D
:103FF00008B100F079FA6D1E6DB2002DF3DC84F883
:104000004460BDE8F04100F0FFB800002DE9F04148
:104010000546002700F0E6FA314E306808B9FFF790
:1040200079FDF06805424BD1C5B3083568070ED05D
:1040300005F00700C0F108000544680707D05020CC
:1040400080F31188BFF34F8FBFF36F8FFEE72DB35F
:104050007068854234D82248103001460C6801E06F
:1040600020460C466168A94202D221680029F7D196
:1040700031688C4224D00768216801606068083785
:10408000411B10290FD96019420708D0502080F336
:104090001188BFF34F8FBFF36F8FFEE710E04160D1
:1040A0006560FFF7EDFD61687068401A7060B26886
:1040B000904200D2B060F06801430020C4E90001E2
:1040C00000F07EFF780707D0502080F31188BFF3FF
:1040D0004F8FBFF36F8FFEE73846BDE8F0810000D9
:1040E0006C00002010B5031F4FF080741C601B1F74
:1040F00021F001011960191F044B0B6014390A608B
:10410000091F6FF0020244380A6010BD553F0008D5
:10411000D0E9013201699A60D0E901235A604A6806
:10412000824201D182684A60002202610868401E12
:104130000860086870470000034B036003F15C00EF
:104140000860802010607047A8080020044B0360BE
:1041500003F15C0008604FF480701060704700004D
:10416000040B002000F108014FF0FF32C0E90112FA
:10417000C160016100210160704700210161704749
:1041800030B50B685A1C02D000F1080202E0026947
:1041900004E02246546825689D42FAD953684B6072
:1041A00099608A60516008610168491C016030BDF6
:1041B00042684A6093688B609368596091600861B7
:1041C0000168491C01607047502080F31188BFF3DB
:1041D0004F8FBFF36F8F0A494868401C4860012821
:1041E0000CD10848006810F0FF0F07D0502080F372
:1041F0001188BFF34F8FBFF36F8FFEE7704700004A
:104200008400002004ED00E00849486828B1401E01
:10421000486001D180F311887047502080F31188E5
:10422000BFF34F8FBFF36F8FFEE7000084000020C5
:1042300070B5002827D0144DA0F108046168E86823
:10424000014207D1502080F31188BFF34F8FBFF395
:104250006F8FFEE722683AB1502080F31188BFF3D8
:104260004F8FBFF36F8FFEE78143616000F0BAF9B3
:1042700060686968084468602046FFF701FDBDE892
:10428000704000F09DBE70BD6C0000204FF0E0203B
:1042900000210161816105494FF47A720968B1FB1F
:1042A000F2F1491E416107210161704714000020AD
:1042B00010B5FCF715F8114910280ED300F1E020D5
:1042C00090F8F0030A78904207D2502080F31188CA
:1042D000BFF34F8FBFF36F8FFEE70948006889680F
:1042E00000F4E060884207D9502080F31188BFF3C2
:1042F0004F8FBFF36F8FFEE710BD000084000020DA
:104300000CED00E010B5084B002200BF53F832401E
:104310001CB1521C082AF9D310BD43F8321003EB2C
:10432000C201486010BD00008C02002070B5154627
:104330000E460446FFF748FF94F944100020491C3C
:1043400001D184F8440094F94510491C01D184F846
:104350004500FFF759FFA06B28B92A46314604F102
:10436000240000F0DFF82046BDE87040FFF718BEDB
:1043700010B5020014D00F48806B38B1502080F384
:104380001188BFF34F8FBFF36F8FFEE700F02AF95C
:1043900000211046FFF798FA00F012FE002807D11E
:1043A00005494FF080500860BFF34F8FBFF36F8F08
:1043B00010BD00001800002004ED00E070B50D46AF
:1043C00004000BD095B11E4A906BB8B1502080F319
:1043D0001188BFF34F8FBFF36F8FFEE7502080F33C
:1043E0001188BFF34F8FBFF36F8FFEE7502080F32C
:1043F0001188BFF34F8FBFF36F8FFEE700F0F2F825
:10440000526923685919934204D98B420AD99142BF
:1044100002D807E08B42FAD9881A21600021FFF701
:1044200053FA00E0216000F0CBFD002807D10549D8
:104430004FF080500860BFF34F8FBFF36F8F70BD98
:104440001800002004ED00E070B50546FFF7BCFE43
:104450001E4C05B92568281DFFF75AFEA86A18B139
:1044600005F11800FFF754FEE06A401CE062206886
:10447000854207D1291D1648FFF79AFEE068401CC7
:10448000E06007E02069401E20612846FFF727FB17
:10449000FFF706FDFFF7B8FEE069002814D020689A
:1044A000854211D1A06B38B1502080F31188BFF341
:1044B0004F8FBFF36F8FFEE706494FF080500860C3
:1044C000BFF34F8FBFF36F8F70BD00001800002047
:1044D0006807002004ED00E002498A6A0260496929
:1044E0004160704718000020014901204862704770
:1044F0001800002010B50C4650B109490968183160
:10450000FFF73EFE2046BDE810400121FFF7DCB971
:10451000502080F31188BFF34F8FBFF36F8FFEE7FA
:104520001800002070B514460D4668B10A490968A4
:104530001831FFF73DFE0CB14FF0FF3521462846FC
:10454000BDE87040FFF7C0B9502080F31188BFF379
:104550004F8FBFF36F8FFEE71800002030B587B094
:104560000024039405AA04A903A80494FFF7E4FD1A
:10457000DDE903010094CDE90110002315A11748DE
:10458000059A00F0F4FB164D002868631FD000F078
:1045900079FD012809D0401C19D1502080F31188E1
:1045A000BFF34F8FBFF36F8FFEE7502080F311886A
:1045B000BFF34F8FBFF36F8F4FF0FF3028630120A1
:1045C000E8616C6107B0BDE8304000F045B807B065
:1045D00030BD000049444C4500000000613B00082C
:1045E000180000200248816B491C8163704700005D
:1045F00018000020164810B5816B11B101214162ED
:1046000010BD002141628169124A01E0B9B1491E21
:1046100001EB810352F82330002BF7D001EB81032B
:1046200002EB830202F1080453685B685360A34203
:1046300001D15B685360DA680260816110BD50206F
:1046400080F31188BFF34F8FBFF36F8FFEE7000039
:1046500018000020CC0200201CB537480168374AFA
:10466000914207D1502080F31188BFF34F8FBFF3E1
:104670006F8FFEE700683149491E884207D15020FC
:1046800080F31188BFF34F8FBFF36F8FFEE72C4984
:1046900008780190FF20087008788DF800009DF8D8
:1046A00000009DF8002000F0F000904207D050205C
:1046B00080F31188BFF34F8FBFF36F8FFEE79DF834
:1046C0000000204B00F0500018700720986005E0B3
:1046D0009DF8002052008DF80020401E9DF800201B
:1046E0001206F5D49860032807D0502080F3118873
:1046F000BFF34F8FBFF36F8FFEE74FF440709860AA
:10470000019808700C482030016841F47001016084
:10471000016841F070410160FFF7B8FD002058606A
:10472000FBF7A6FD0848016841F040410160FBF736
:104730008BFD00201CBD000000ED00E071C20F41A8
:1047400000E400E08400002034EF00E010B55020C9
:1047500080F31188BFF34F8FBFF36F8F00F054FBCE
:1047600018B104494FF080500860002080F3118890
:1047700010BD000004ED00E0F8B517460E46050038
:1047800014D0DEB105FB06F05030FFF73FFC04000B
:104790000AD0002084F8460004F150023B4631461E
:1047A00028460094FFF70CFA2046F8BD502080F30D
:1047B0001188BFF34F8FBFF36F8FFEE70020E3E751
:1047C00038B5049D18B153B1CAB181B120E0502071
:1047D00080F31188BFF34F8FBFF36F8FFEE7502038
:1047E00080F31188BFF34F8FBFF36F8FFEE7502028
:1047F00080F31188BFF34F8FBFF36F8FFEE739B19E
:10480000502080F31188BFF34F8FBFF36F8FFEE707
:1048100050241C46012384F846302B460094FFF7B1
:10482000CFF9204638BD000070B50D46040025D0F4
:10483000FFF7CAFCD4E90F20216802FB0011616078
:104840000021A1632168A1600A46D4E90F01401E3E
:1048500000FB0121E16021464FF0FF3001F8440FD9
:10486000487004F110008DB1FFF77CFC04F12400C6
:10487000FFF778FCFFF7C8FC012070BD502080F3E3
:104880001188BFF34F8FBFF36F8FFEE721690029B7
:10489000F0D000F05DFB0028ECD004494FF08050D0
:1048A0000860BFF34F8FBFF36F8FE3E704ED00E0C5
:1048B0002DE9FF4782B01D468A464FF000080400EC
:1048C00003D0BAF1000F08D011E0502080F3118816
:1048D000BFF34F8FBFF36F8FFEE7206C38B15020CE
:1048E00080F31188BFF34F8FBFF36F8FFEE7022D68
:1048F0000AD1E06B012807D0502080F31188BFF364
:104900004F8FBFF36F8FFEE700F062FA3F4F4FF01B
:1049100000094FF0805648B9049838B1502080F310
:104920001188BFF34F8FBFF36F8FFEE7FFF74CFC8B
:10493000A06BE16B884207D3022D05D00498D0B15B
:10494000B8F1000F1AD01EE02A4651462046FFF764
:1049500090F8616A19B104F1240000F0F9FA20B16D
:104960003E60BFF34F8FBFF36F8FFFF74DFC012009
:1049700006B0BDE8F087FFF747FC22E06846FFF786
:10498000ABFD4FF00108FFF73FFCFFF72BFEFFF7F1
:104990001BFC94F94400401C01D184F8449094F924
:1049A0004500401C01D184F84590FFF72DFC04A977
:1049B000684600F075F930B12046FFF7F1FA00F0D3
:1049C000FFFA0020D4E7FFF7FFFBA06BE16B884202
:1049D00013D1FFF719FC04F110000499FFF78AFDC9
:1049E0002046FFF7DDFA00F0EBFA00289ED13E608A
:1049F000BFF34F8FBFF36F8F98E7FFF705FC20469B
:104A0000FFF7CEFA00F0DCFA90E7000004ED00E0DA
:104A10002DE9F0471F4690468946040003D0B9F1BE
:104A2000000F08D011E0502080F31188BFF34F8FA2
:104A3000BFF36F8FFEE7206C38B1502080F31188F0
:104A4000BFF34F8FBFF36F8FFEE7022F0AD1E06BEA
:104A5000012807D0502080F31188BFF34F8FBFF398
:104A60006F8FFEE7FFF724FC5020EFF3118680F3F1
:104A70001188BFF34F8FBFF36F8FA06BE16B88423C
:104A800006D3022F04D0002086F31188BDE8F087FA
:104A900094F945503A4649462046FEF7EAFF681C1D
:104AA00004D06D1C84F845500120EDE7606A0028B1
:104AB000FAD004F1240000F04BFA0028F4D0B8F149
:104AC000000FF1D00121C8F80010EDE72DE9F747FC
:104AD000002683B08A46040003D0BAF1000F08D044
:104AE00011E0502080F31188BFF34F8FBFF36F8F19
:104AF000FEE7206C38B1502080F31188BFF34F8F50
:104B0000BFF36F8FFEE700F063F9DFF8F4804FF03A
:104B100000094FF0805748B9059838B1502080F30C
:104B20001188BFF34F8FBFF36F8FFEE7FFF74CFB8A
:104B3000A56BC5B151462046FEF788FF6D1EA563E3
:104B4000206950B104F1100000F002FA28B1C8F851
:104B50000070BFF34F8FBFF36F8FFFF755FB01203E
:104B600006B0BDE8F087059808B11EB106E0FFF772
:104B70004BFB27E06846FFF7AFFC0126FFF744FB3D
:104B8000FFF730FDFFF720FB94F94400401C01D1F2
:104B900084F8449094F94500401C01D184F8459074
:104BA000FFF732FB05A9684600F07AF80028204696
:104BB0000AD0FFF7F5F900F003FA2046FFF7A2F854
:104BC0000028B3D00020CBE7FFF79CF890B104F1A8
:104BD00024000599FFF78EFC2046FFF7E1F900F06D
:104BE000EFF90028A2D1C8F80070BFF34F8FBFF3D0
:104BF0006F8F9BE72046FFF7D3F900F0E1F995E7C7
:104C000004ED00E02DE9F04790468946040003D00A
:104C1000B9F1000F08D011E0502080F31188BFF3E4
:104C20004F8FBFF36F8FFEE7206C38B1502080F3B9
:104C30001188BFF34F8FBFF36F8FFEE7FFF738FB8D
:104C40005020EFF3118680F31188BFF34F8FBFF32D
:104C50006F8FA76BF7B194F9445049462046FEF791
:104C6000F5FE7F1EA763681C04D06D1C84F84450B9
:104C7000012010E020690028FAD004F1100000F0B3
:104C800067F90028F4D0B8F1000FF1D00121C8F87D
:104C90000010EDE7002086F31188BDE8F0870000E2
:104CA0002DE9F0410C46050011D0C4B1FFF78CFA94
:104CB000174B5A696E682068911B471C17D02F68E4
:104CC0009B6A9F4219D0964217D8012410E05020C9
:104CD00080F31188BFF34F8FBFF36F8FFEE7502033
:104CE00080F31188BFF34F8FBFF36F8FFEE700246F
:104CF000FFF78AFA2046BDE8F081884205D9401ABC
:104D000020602846FFF7E8FBF1E700202060DCE7A1
:104D1000180000202DE9FF5F8346DDE90E879946E4
:104D200016468A469000FFF771F905001CD05C20FA
:104D3000FFF76CF9040014D00020256384F85900B3
:104D4000CDE90240CDE900874B46324651465846F0
:104D5000FEF747FF2046FEF7E5FD012004B0BDE861
:104D6000F09F2846FFF764FA4FF0FF30F6E7F0B502
:104D700085B0DDE90B640A9DA6B1DCB15C27009724
:104D80002663022684F85960002604AFCDE9024666
:104D9000CDE90057FEF725FF2046FEF7C3FD049836
:104DA00005B0F0BD502080F31188BFF34F8FBFF3E3
:104DB0006F8FFEE7502080F31188BFF34F8FBFF352
:104DC0006F8FFEE701480068704700001800002060
:104DD0000548C16919B1806B18B1002070470120E6
:104DE0007047022070470000180000200148406909
:104DF000704700001800002010B5FFF759FA01486D
:104E0000406910BD180000202DE9F0412E4C00270C
:104E1000A06B40B1206A401C2062606A00B101278B
:104E20003846BDE8F0816669761C666113D160681A
:104E3000006838B1502080F31188BFF34F8FBFF363
:104E40006F8FFEE76068A1686160A060A06A401C87
:104E5000A062FFF725F8206BDFF87080864209D347
:104E60006068006880B16068C068C568686886422C
:104E70000DD220632068C06A00EB800158F8210041
:104E80000128CAD90127C8E74FF0FF30F1E7281DF4
:104E9000FFF73EF9A86A18B105F11800FFF738F9D5
:104EA000E86AA169884200D9A06100EB800108EBA3
:104EB0008100291DFFF77CF9E86A2168C96A8842E8
:104EC000CED30127CCE7000018000020CC02002040
:104ED00070B504004FF0000133D01B4D28688442A8
:104EE00007D0502080F31188BFF34F8FBFF36F8F2F
:104EF000FEE7206D38B1401E2065E36CE26A9A42FD
:104F00001FD040B11DE0502080F31188BFF34F8FB8
:104F1000BFF36F8FFEE7201DFFF7FAF8E06CE06249
:104F2000C0F13800A061E06AA969884200D9A8618F
:104F3000064900EB800001EB8000211DFFF738F9E6
:104F40000121084670BD000018000020CC0200209E
:104F500070B5C068C46854B104F118000646FFF784
:104F6000D7F8144DA86B50B13146134815E05020C6
:104F700080F31188BFF34F8FBFF36F8FFEE7201DC3
:104F8000FFF7C6F8E06AA969884200D9A8610B4911
:104F900000EB800001EB8000211DFFF709F9E06ABA
:104FA0002968C96A884202D90120686270BD002060
:104FB00070BD00001800002054070020CC02002023
:104FC0002DE9F0472C4D00242746A86B38B1FFF798
:104FD000FBF8A86B401EA863A86B40B146E05020C8
:104FE00080F31188BFF34F8FBFF36F8FFEE72969FE
:104FF000224E0120D1B3A6F5916980463068E0B118
:10500000F068C46804F11800FFF782F8201DFFF76C
:105010007FF8E06AA969884200D9A86100EB8001A5
:1050200009EB8100211DFFF7C3F8E06A2968C96A0E
:105030008842E3D3C5F82480E0E70CB1FEF730FFE7
:105040002C6A4CB14FEA0806FFF7DEFE00B16E6233
:10505000641EF9D100202862686A38B10849012726
:1050600038070860BFF34F8FBFF36F8FFFF7CCF89F
:105070003846BDE8F08700001800002054070020E3
:1050800004ED00E010B586B0FEF7B4FC114CA0684A
:10509000B8B100200390049005AA04A903A8FFF763
:1050A00055F8DDE9032102208DE8070000230AA15D
:1050B0000B48059AFFF75BFEE06010B106B00120D7
:1050C00010BD502080F31188BFF34F8FBFF36F8F57
:1050D000FEE7000054000020546D722053766300F8
:1050E0007D3F00082DE9FF411E46134602000A9D40
:1050F0004FF0000016D0144CA768002F0FD0CDE958
:1051000000130292062917DAFFF762FE02284FF019
:1051100000030FD000226946A068FFF7C9FB04B066
:10512000BDE8F081502080F31188BFF34F8FBFF3AB
:105130006F8FFEE72A46EEE700233246694638467F
:10514000FFF766FCEBE70000540000204FF04070D2
:10515000E1EE100A704700006852000800000000ED
:10516000000000000000000000000000000200003D
:105170001800000000000000000000000203040509
:10518000060708090A0B0C0D0E0F1010010203048C
:1051900005060708090A0B0C0D0E0F100000000091
:1051A00000000000010203040607080900000000D7
:1051B0000102030474520008000000000000000017
:1051C00000000000000000000004000030000000AB
:1051D00000000000000000008052000800000000F5
:1051E00000000000000000000000000000020000BD
:1051F0003000000000000000000000008C52000899
:10520000000000000000000000000000000000009E
:10521000000200003000000000000000000000005C
:10522000985200080000000000000000000000008C
:10523000000000000002000030000000000000003C
:1052400000000000A852000800000000000000005C
:10525000000000000000000000020000300000001C
:10526000000000000000000064656661756C745405
:1052700061736B005461736B5F496E697400000069
:105280005461736B5F43616E000000005461736B87
:105290005F416463000000005461736B5F4D6F6E8B
:1052A00069746F72000000005461736B5F504300BB
:1052B000D052000800000020A4000000C401000833
:1052C00074530008A400002084350000E0010008A9
:1052D00000000000000000000100000010000000BD
:1052E0000000000000127A00000000000000000032
:1052F00000000000000000000000000000000000AE
:10530000000000000000000000000000000000009D
:10531000000000000000000000000000000000008D
:10532000000000000000000000000000000000007D
:10533000000000000000000000000000000000006D
:10534000000000000000000000000000000000005D
:105350000000000000000000AAAAAAAA00000000A5
:10536000000000000000000001000000000000003C
:045370000000000039
:040000050800018965
:00000001FF
